:1000000008308A00992D0000FF00030E8301A10033
:100010000A08A0008A010408A2007708A300780853
:10002000A4007908A5007A08A6007B08A70083131E
:1000300083120B1E1D288B183028220884002308E9
:10004000F7002408F8002508F9002608FA00270818
:10005000FB0020088A00210E8300FF0E7F0E09009E
:100060008A110A1600280A108A100A11820712340F
:10007000013410340134FF34FF34FF3410340434BD
:100080007134113402340034003401340234003449
:1000900001340A108A100A1182070934023422340A
:1000A0000034013401340034A034053409340434FC
:1000B0000034003401340334013401340034093491
:1000C0002134013400340034013422340034323419
:1000D0000734053481340334103400340A340A10F0
:1000E0008A100A11820704340334093404340A10D4
:1000F0008A100A118207763403345034003468348D
:100100000034693400346C340034693400342034F1
:1001100000342D3400342D34003470340034733402
:1001200000342034003453340034653400346D34EA
:10013000003469340034633400346F3400346E3476
:10014000003464340034753400346334003474345F
:1001500000346F340034723400347334003420348B
:1001600000342D34003420340034413400347334EE
:1001700000346934003461340034203400345034A5
:100180000034723400346F34003464340034753415
:10019000003463340034743400342034003449347F
:1001A00000346E3400346E3400346F3400347634EE
:1001B00000346134003474340034693400346F34F2
:1001C00000346E3400342034003443340034653459
:1001D00000346E34003474340034723400346534C6
:1001E00000340A108A100A11F83E03188A0A8200A5
:1001F0004634033450340034443400344934003439
:100200005534003453340034423400344434003420
:100210003134003431340034203400342C34003490
:100220002034003444340034313400343134003468
:1002300020340034463400346934003472340034DD
:100240006D34003477340034613400347234003457
:1002500065340034203400345634003465340034BE
:100260007234003473340034693400346F34003431
:100270006E34003420340034313400340A148A10CF
:100280000A118207083403345834003457340034D8
:100290004C3400340A148A100A118207443444345E
:1002A0005234203400340A148A100A11820744346C
:1002B0006134743461344C3465346E343D342534E7
:1002C0007834203400340A148A100A118207433427
:1002D00044345234203400340A148A100A1182073C
:1002E000533444345234203400340A148A100A112E
:1002F0008207213444345334283425347834293463
:1003000000340A148A100A1182070D340A340D349D
:100310000A3425346434203400340A148A100A1153
:1003200082075F34533441344534203400340A1496
:100330008A100A1182075F3453344534453420341F
:1003400000340A148A100A1182075F3453344D3482
:10035000203400340A148A100A11820753345234AC
:1003600045345134203400340A148A100A118207AB
:100370004334523445345134203400340A148A1042
:100380000A11820745345234453451342034003444
:100390000A148A100A1182073F345234453451340A
:1003A0003D3425347834203400340A148A100A117C
:1003B00082074734653474345F34533474346134A1
:1003C00075347334203400340A148A100A118207F9
:1003D00043346C346534613472345F34463465348C
:1003E00061347434753472346534203400340A1442
:1003F0008A100A11FE3E03188A0A820053346534BB
:1004000074345F34663465346134743475347234F2
:100410006534203400340A108A140A1182075334D8
:10042000653474345F344134643464347234653414
:1004300073347334203400340A108A140A1182078A
:100440004734653474345F3444346534733463340E
:1004500072346934703474346F347234203400343C
:100460000A108A140A1182075334653474345F34D5
:10047000443465347334633472346934703474349E
:100480006F347234203400340A108A140A1182073F
:100490004734653474345F3443346F346E346634B7
:1004A00069346734753472346134743469346F3448
:1004B0006E34203400340A108A140A11820753342F
:1004C000653474345F3443346F346E346634693465
:1004D0006734753472346134743469346F346E3413
:1004E000203400340A108A140A1182074734653414
:1004F00074345F3449346E34743465347234663421
:10050000613463346534203400340A108A140A11CB
:1005100082075334653474345F3449346E34743430
:1005200065347234663461346334653420340034A5
:100530000A108A140A118207533479346E346334F2
:1005400068345F344634723461346D346534203439
:1005500000340A108A140A1182073F34533452348B
:10056000453451343D3425347834203400340A1075
:100570008A140A1182075334443452343D342534EA
:100580007834203400340A108A140A1182073F3468
:10059000533444345234203400340A108A140A117B
:1005A00082073F34443452343D3425347834203487
:1005B00000340A108A140A11820721344C3454344E
:1005C0003D3425347834203400340A108A140A115A
:1005D00082073F344C3454343D342534783420344D
:1005E00000340A108A140A11820744344934523400
:1005F0003D34003400000A148A140A11023E031824
:100600008A0A820053344134453450342034003453
:100610000C1E082B83162C088312990000348316B5
:100620002708F700F708831203191B2B0130770204
:1006300003191B2B482B0030831688008610831269
:1006400086148316270B292B0613831206172C2BCF
:100650008316061383120613831628088312880054
:1006600008308316A9002908A903003A031D332B7B
:1006700006118312061183160611831206158316BE
:10068000270B462B0613831206138316472B831260
:100690000034FF3083168800A201210822020318CB
:1006A000622B86108312861083162008220784008E
:1006B000831208088000831686108312861483161E
:1006C000A20A4D2B831200348316AB1B792B0F30FB
:1006D000F7002A0EF7050A3077020318722B303024
:1006E000F707742B2B08F7077708AC008312082351
:1006F00083160F30AA050A302A020318812B3030E6
:10070000832BAB132B08AA072A08AC0083120823FB
:100710000034AF01B001AD01AC08031D902B2B14C8
:10072000AC08031DA02BE10161088D21E10AF7004F
:100730008316AC008312082305306102031D942B3D
:1007400001308316A700D030A80083120F23831630
:10075000A7018030A80083120F23AC08031DB12B22
:100760002B14AC08031DC12BE10161089721E10A9C
:10077000F7008316AC008312082305306102031DC5
:10078000B52B01308316A700D830A80083120F23A1
:100790008316A7010130A80083120F23AC08031DA4
:1007A000D22B2B14AC08031DE22BE1016108A1211F
:1007B000E10AF7008316AC008312082304306102BB
:1007C000031DD62B01308316A700F330A800831237
:1007D0000F238316A7011E30A80083120F23831650
:1007E000A7010B30A80083120F2300342C08053C0E
:1007F000031CFB2B2B142C08053C031C092C533029
:100800008316AC00831208235F308316AC0083127A
:10081000082383162508F700F70883120319252CEF
:100820000130770203193E2C023077020319572C4E
:10083000033077020319702C043077020319892CD6
:10084000053077020319A22CBB2C2C08053C031C95
:100850002A2C2B142C08053C031C3D2C43308316FA
:10086000AC00831208234F308316AC008312082398
:1008700020308316AC0083120823E02C2C08053CA2
:10088000031C432C2B142C08053C031C562C433012
:100890008316AC008312082349308316AC00831200
:1008A000082320308316AC0083120823E02C2C0888
:1008B000053C031C5C2C2B142C08053C031C6F2CE2
:1008C00045308316AC00831208234F308316AC00EA
:1008D0008312082320308316AC0083120823E02CF7
:1008E0002C08053C031C752C2B142C08053C031C00
:1008F000882C45308316AC008312082349308316B8
:10090000AC008312082320308316AC008312082326
:10091000E02C2C08053C031C8E2C2B142C08053CC9
:10092000031CA12C4D308316AC00831208234F30DA
:100930008316AC008312082320308316AC00831288
:100940000823E02C2C08053C031CA72C2B142C0896
:10095000053C031CBA2C4D308316AC0083120823CF
:1009600049308316AC008312082320308316AC0074
:1009700083120823E02C2C08053C031CC02C2B14EC
:100980002C08053C031CDF2C3F308316AC0083127F
:10099000082328308316AC00831208238316250809
:1009A000AA005730AB008312642329308316AC00B1
:1009B0008312082320308316AC0083120823E02C16
:1009C000403083162507A6000130A7002608A8009E
:1009D00083120F238316A7010130A80083120F236F
:1009E00000342C08043C031CF62C2B142C08043C6B
:1009F000031C0B2D8316A10121088312F1228316FB
:100A0000A10AF700AC0083120823043083162102E8
:100A1000031DFC2C8312831620088400801F262DC2
:100A200083122C08043C031C162D2B142C08043CA8
:100A3000031C242D49308316AC0083120823203078
:100A40008316AC00831208233A2D831683122C08D8
:100A5000043C031C2C2D2B142C08043C031C3A2DA5
:100A60004F308316AC008312082320308316AC006D
:100A7000831208232C08043C031C3F2D2B142C0844
:100A8000043C031C522D54308316AC0083120823FF
:100A90004F308316AC00831208233D308316AC0020
:100AA0008312082383162008840000081F39F700EA
:100AB000F70883120319692D0130770203197D2D80
:100AC000023077020319912D033077020319A52D07
:100AD000B92D2C08043C031C6E2D2B142C08043C4F
:100AE000031C7C2D44308316AC0083120823203075
:100AF0008316AC0083120823CC2D2C08043C031C65
:100B0000822D2B142C08043C031C902D4930831695
:100B1000AC008312082320308316AC008312082314
:100B2000CC2D2C08043C031C962D2B142C08043CC3
:100B3000031CA42D45308316AC00831208232030FB
:100B40008316AC0083120823CC2D2C08043C031C14
:100B5000AA2D2B142C08043C031CB82D3F308316FF
:100B6000AC008312082320308316AC0083120823C4
:100B7000CC2D2C08073C031CBE2D2B142C08073C45
:100B8000031CC72D07308316AC008312082383167D
:100B9000A5018312F623CC2D2C08043C031CD12D77
:100BA0002B142C08043C031C002E02308316200753
:100BB0008400840A0008A20084030008A1007730A2
:100BC000AC008312082356308316AC00831208232E
:100BD0003D308316AC008312082383162208AA0036
:100BE0005730AB008312642383162108AA005730C4
:100BF000AB008312642320308316AC0083120823D9
:100C00002C08043C031C052E2B142C08043C031C4C
:100C1000342E0430831620078400840A0008A200C2
:100C200084030008A1007730AC0083120823493008
:100C30008316AC00831208233D308316AC00831268
:100C4000082383162208AA005730AB0083126423BE
:100C500083162108AA005730AB008312642320308A
:100C60008316AC00831208232C08043C031C392E85
:100C70002B142C08043C031C682E06308316200716
:100C80008400840A0008A20084030008A1007730D1
:100C9000AC00831208234C308316AC008312082367
:100CA0003D308316AC008312082383162208AA0065
:100CB0005730AB008312642383162108AA005730F3
:100CC000AB008312642320308316AC008312082308
:100CD00000340230831621078400840A0008A30030
:100CE00084030008A20080388312AF002C08033C64
:100CF000031C7B2E2B142C08033C031C902E831604
:100D0000A20122088312FA228316A20AF700AC007D
:100D100083120823053083162202031D812E8312BD
:100D200000342C08053C031C962E2B142C08053C83
:100D3000031CB52E8316A20122088312D922831622
:100D4000A20AF700AC0083120823043083162202A3
:100D5000031D9C2E2108AA005730AB008312642388
:100D600020308316AC008312082383162108F70075
:100D70000230770283120319EE2E04307702031932
:100D8000EF2E063077020319F02E08307702031990
:100D9000F12E0A3077020319F22E0C307702031974
:100DA000F32E0E3077020319F42E10307702031958
:100DB000F52E123077020319F62E1430770203193C
:100DC000F72E163077020319F82E1A30770203191E
:100DD000F92E1E3077020319FA2EFB2E2E2F2E2FFE
:100DE0002E2F2E2F2E2F2E2F2E2F2E2F2E2F2E2F1B
:100DF0002E2F2E2F2E2F2C08073C031C002F2B14D8
:100E00002C08073C031C092F07308316AC00831203
:100E100008232C08053C031C0E2F2B142C08053C22
:100E2000031C2D2F8316A20122088312E5228316AC
:100E3000A20AF700AC0083120823043083162202B2
:100E4000031D142F2108AA005730AB00831264231E
:100E500020308316AC00831208232E2F003401307B
:100E60008316A700831261088316A80083120F233C
:100E700001308316A700F030A80083120F238316D9
:100E8000A701A80183120F238316A701A8018312CB
:100E90000F2301308316A700FA30A80083120F2316
:100EA0002C08033C031C552F2B142C08033C031C5B
:100EB000632F5A308316AC00831208232030831628
:100EC000AC008312082300343508F80134020318FB
:100ED0006C2F3408F700782FF7010830B600B40DF6
:100EE000F70D350877020318F700F80DB60B6F2FD2
:100EF00000343208F700B21B812F331D942F2030AD
:100F0000862FF709F70A7708B2002D30F800A801FC
:100F10008B1BA8178B1378088316AC008312082349
:100F2000A81B8B17331DB3153208B4006430B5000D
:100F300064277708B20078083030031DA62F3318D5
:100F4000B42FB319B42F331A2030A82FB311331292
:100F5000F807A8018B1BA8178B1378088316AC0021
:100F600083120823A81B8B173208B4000A30B5007F
:100F700064277708B20078083030031DC32FB319F7
:100F8000CF2F331A2030F807A8018B1BA8178B131B
:100F900078088316AC0083120823A81B8B17303007
:100FA000B207A8018B1BA8178B1332088316AC005D
:100FB00083120823A81B8B178A150A12FB2D3130C8
:100FC000840000080319F32F0130F800F701F70B34
:100FD000E72FF80BE62F4A30F700F70BED2F000054
:0C0FE0000000800BE42F8A150A120D2E71
:1010000083162414063021078400840A0008FA009D
:1010100084030008A2007A08A3000230210784009C
:10102000840A0008A60084030008A5002608FA0127
:10103000F7007A08031D2228013077028312031972
:10104000352883167A08031D2B2802307702831275
:101050000319622883167A08031D342803307702A7
:10106000831203198F28831669292C08033C031C5B
:101070003A282B142C08033C031C53288316A50183
:1010800025088A1183124A218A158316A50AF700BA
:10109000AC008A11831208238A15043083162502B6
:1010A000031D402883128316A308031D5B28220812
:1010B000123C03185E28A3011230A20001308312F3
:1010C000B000BA292C08033C031C67282B142C08F9
:1010D000033C031C80288316A50125088A1183126E
:1010E00063218A158316A50AF700AC008A118312C2
:1010F00008238A15043083162502031D6D288312E8
:101100008316A308031D88282208223C03188B2875
:10111000A3012230A20002308312B000BA292C08A9
:10112000033C031C94282B142C08033C031CC928E3
:101130000230831621078400840A0008A600840375
:101140000008A5000F39A70026080039A800A9014A
:1011500029088A118312B7228A158316A90AF70073
:10116000AC008A11831208238A15043083162902E1
:10117000031DA8282708AA005730AB008A11831244
:1011800064238A1520308316AC008A118312082349
:101190008A150230831621078400840A0008A600FD
:1011A00084030008A5000F39F70026080039FA006B
:1011B0007A08031DE028F70883120319FC28831618
:1011C0007A08031DE92801307702831203190A29DE
:1011D00083167A08031DF22802307702831203195E
:1011E000182983167A08031DFB280330770283121F
:1011F00003192629831634290330B0008316A30867
:10120000031D06292208043C03180929A301043000
:10121000A20066290430B0008316A308031D142918
:101220002208763C03181729A3017630A20066290C
:101230000530B0008316A308031D22292208463C6E
:1012400003182529A3014630A20066290630B00004
:101250008316A308031D30292208083C03183329EC
:10126000A3010830A200662983122C08043C031C49
:101270003A292B142C08043C031C452907308316FB
:10128000AC008A11831208238A152C08043C031C25
:101290004A292B142C08043C031C63298316A5013E
:1012A00025088A118312C3228A158316A50AF7001E
:1012B000AC008A11831208238A1505308316250293
:1012C000031D502983128316241066298312BA291C
:1012D0008316241083122C08043C031C70292B1441
:1012E0002C08043C031C7B2907308316AC008A11B0
:1012F000831208238A152C08053C031C80292B1413
:101300002C08053C031CB3290230831621078400F6
:10131000840A0008A60084030008A5002608A70088
:10132000A801A90129088A118312CD228A158316E2
:10133000A90AF700AC008A11831208238A15043029
:1013400083162902031D92292708AA005730AB00F3
:101350008A11831264238A1520308316AC008A1107
:10136000831208238A158316A5018A118312F62396
:101370008A15BA298316241CC4298312AD01831649
:1013800022088312AE0083168312003401308316C4
:10139000200784000008F700F70883120319F929D1
:1013A000013077020319182A033077020319372A0C
:1013B000053077020319562A0630770203197C2A72
:1013C000073077020319A02A083077020319BF2AD1
:1013D000093077020319DE2A0A3077020319FD2A41
:1013E0000B30770203191C2B0C30770203193B2BAF
:1013F0005A2B2C08053C031CFE292B142C08053CF9
:10140000031C172A8316A10121088A118312D521F2
:101410008A158316A10AF700AC008A1183120823EB
:101420008A150A3083162102031D042A83129C2B7D
:101430002C08053C031C1D2A2B142C08053C031CFE
:10144000362A8316A10121088A118312E4218A1504
:101450008316A10AF700AC008A11831208238A15AB
:101460000E3083162102031D232A83129C2B2C0885
:10147000053C031C3C2A2B142C08053C031C552A54
:101480008316A10121088A118312F7218A15831678
:10149000A10AF700AC008A11831208238A150C30C8
:1014A00083162102031D422A83129C2B2C08053C23
:1014B000031C5B2A2B142C08053C031C742A83167E
:1014C000A10121088A1183120B228A158316A10A11
:1014D000F700AC008A11831208238A150C3083169A
:1014E0002102031D612A831283162008A1008A119C
:1014F000831269268A159C2B2C08053C031C812A23
:101500002B142C08053C031C9A2A8316A1012108E0
:101510008A1183121C228A158316A10AF700AC00D7
:101520008A11831208238A150F3083162102031DA6
:10153000872A831283162008A100831200209C2B87
:101540002C08053C031CA52A2B142C08053C031C65
:10155000BE2A8316A10121088A11831230228A151E
:101560008316A10AF700AC008A11831208238A159A
:101570000F3083162102031DAB2A83129C2B2C08EB
:10158000053C031CC42A2B142C08053C031CDD2A33
:101590008316A10121088A11831244228A15831619
:1015A000A10AF700AC008A11831208238A151230B1
:1015B00083162102031DCA2A83129C2B2C08053C8A
:1015C000031CE32A2B142C08053C031CFC2A83165D
:1015D000A10121088A1183125B228A158316A10AB0
:1015E000F700AC008A11831208238A151230831683
:1015F0002102031DE92A83129C2B2C08053C031CA5
:10160000022B2B142C08053C031C1B2B8316A10159
:1016100021088A11831272228A158316A10AF70003
:10162000AC008A11831208238A150E30831621021A
:10163000031D082B83129C2B2C08053C031C212B1B
:101640002B142C08053C031C3A2B8316A1012108FE
:101650008A11831285228A158316A10AF700AC002D
:101660008A11831208238A150E3083162102031D66
:10167000272B83129C2B2C08053C031C402B2B147E
:101680002C08053C031C592B8316A10121088A1143
:10169000831298228A158316A10AF700AC008A11DA
:1016A000831208238A150C3083162102031D462B52
:1016B00083129C2B2C08073C031C5F2B2B142C083B
:1016C000073C031C6A2B07308316AC008A11831277
:1016D00008238A152C08053C031C6F2B2B142C089F
:1016E000053C031C9B2B0130831620078400000857
:1016F000A100A20122088A118312A9228A15831649
:10170000A20AF700AC008A11831208238A1506305A
:1017100083162202031D7A2B2108AA005730AB0042
:101720008A11831264238A1520308316AC008A1133
:10173000831208238A159C2B003401308316A700DE
:101740004030A8008A1183120F238A156130831656
:10175000A0000130A1008A11831249238A152C08A8
:10176000033C031CB42B2B142C08033C031CDD2B63
:101770004C308316AC008A11831208238A1554302A
:101780008316AC008A11831208238A153D30831614
:10179000AC008A11831208238A1561088316AA00F7
:1017A0005730AB008A11831264238A1520308316C8
:1017B000AC008A11831208238A15E11FDF2B611CFC
:1017C0008A2DE11E892D01308316A700A8018A11F8
:1017D00083120F238A1563308316A0000130A10005
:1017E0008A11831249238A152C08023C031CF92B09
:1017F0002B142C08023C031C222C53308316AC0003
:101800008A11831208238A1545308316AC008A1189
:10181000831208238A153D308316AC008A11831287
:1018200008238A1563088316AA005730AB008A1173
:10183000831264238A1520308316AC008A11831228
:1018400008238A1501308316A700F030A8008A11FA
:1018500083120F238A1563308316A0001030A10075
:101860008A11831249238A152C08023C031C392C47
:101870002B142C08023C031C622C44308316AC0051
:101880008A11831208238A154C308316AC008A1102
:10189000831208238A153D308316AC008A11831207
:1018A00008238A1564088316AA005730AB008A11F2
:1018B000831264238A1520308316AC008A118312A8
:1018C00008238A1501308316A700F130A8008A1179
:1018D00083120F238A1501308316A700F230A80067
:1018E0008A1183120F238A1501308316A700A800DE
:1018F0008A1183120F238A1501308316A700F13055
:10190000A8008A1183120F238A1501308316A700BD
:10191000F230A8008A1183120F238A156408083C4C
:10192000031D832D0230F4007408093C031CB52C00
:10193000AC08031D9C2C2B14AC08031DB32C633086
:101940007407840000088316A000AA005730AB007B
:101950008A11831264238A1520308316AC008A1101
:10196000831208238A15F40A942C6530F300730857
:101970008316A0008A118312F1248A15730884004B
:1019800000086039F700F70EF70C0730F705770805
:101990000319D32C013077020319F72C0230770298
:1019A0000319162D352D2C08023C031CD82C2B14A2
:1019B0002C08023C031CF12C8316A00120088A117C
:1019C0008312AA218A158316A00AF700AC008A1197
:1019D000831208238A15053083162002031DDE2C8E
:1019E000831273088316A0008312C621822D2C084F
:1019F000023C031CFC2C2B142C08023C031C152D50
:101A00008316A00120088A118312B4218A15831637
:101A1000A00AF700AC008A11831208238A1505304A
:101A200083162002031D022D8312822D2C08023CF6
:101A3000031C1B2D2B142C08023C031C342D831675
:101A4000A00120088A118312BE218A158316A00ADC
:101A5000F700AC008A11831208238A15053083161B
:101A60002002031D212D8312822D2C08043C031C0F
:101A70003A2D2B142C08043C031C452D07308316EB
:101A8000AC008A11831208238A152C08023C031C1F
:101A90004A2D2B142C08023C031C7B2D7308840058
:101AA00000086039F700770E8316A200A20C0730F9
:101AB000A205A30123088A118312C8218A1583165F
:101AC000A30AF700AC008A11831208238A15053097
:101AD00083162302031D5A2D2208AA005730AB009B
:101AE0008A11831264238A1520308316AC008A1170
:101AF000831208238A158316A5018A118312F623FF
:101B00008A15822D892D8316A5018A118312F62349
:101B10008A15982D61081E39003A0319982D61081D
:101B20001E398316A000A1008A11831291268A15FE
:101B3000003484011F308305063083169F000C306B
:101B4000990026309800903083129800A901FF3048
:101B5000AA002B1083168613831286130130831676
:101B6000860000308800FF308312880083168610BC
:101B70008312861483160611831206158316061324
:101B80008312061383160612831206120B138B138D
:101B90008B1BC72D8316011383120B168B10C030BD
:101BA0008B0405080739AC002C08073C031CD92D11
:101BB0002B142C08073C031C092EB10131088A1193
:101BC00081218A15B10AF700A8018B1BA8178B1376
:101BD00077088316AC008A11831208238A15A81B84
:101BE0008B1704303102031DDE2D2C08B200183093
:101BF000B3008A11792F8A15A8018B1BA8178B13A4
:101C000020308316AC008A11831208238A15A81B82
:101C10008B170130B1008A11DF2F8A158316061445
:101C20000030831206180130003A031D222EA8014D
:101C30008B1BA8178B130A168A118B140A128A158C
:081C4000A81B8B17222E630084
:102000008316061483120618212F00302B18013076
:10201000003A03191D2800302B180130E1000D3063
:102020008316AC000A12831208230A160A3083169C
:10203000AC000A12831208230A162B1001308316F3
:10204000A700F430A8000A1283120F230A165C308E
:102050008316A0000230A1000A12831249230A1637
:102060005C08DE005D08DF00AC08031D38282B1477
:10207000AC08031D702849308316AC000A12831285
:1020800008230A1652308316AC000A128312082362
:102090000A163D308316AC000A12831208230A1672
:1020A0005E088316AA005730AB000A12831264231D
:1020B0000A162C308316AC000A12831208230A1663
:1020C0005F088316AA005730AB000A1283126423FC
:1020D0000A1620308316AC000A12831208230A164F
:1020E0005E1F94282C08073C031C77282B142C080F
:1020F000073C031C902842308316AC000A1283125E
:1021000008230A1652308316AC000A1283120823E1
:102110000A1620308316AC000A12831208230A160E
:102120000A1289230A16202FDE1FB5282C08013C2D
:10213000031C9B282B142C08013C031CB42853308F
:102140008316AC000A12831208230A164330831642
:10215000AC000A12831208230A1620308316AC0042
:102160000A12831208230A16202F5E1CDB282C0873
:10217000033C031CBC282B142C08033C031CD5284F
:1021800043308316AC000A12831208230A164F301C
:102190008316AC000A12831208230A162030831615
:1021A000AC000A12831208230A160A128A159D230C
:1021B0000A168A11202FDE1CC02E2C08033C031C9B
:1021C000E2282B142C08033C031CFB284330831605
:1021D000AC000A12831208230A1649308316AC0099
:1021E0000A12831208230A1620308316AC000A1242
:1021F000831208230A1601308316A7004130A80075
:102200000A1283120F230A165C308316A0000130D5
:10221000A1000A12831249230A162C08013C031C50
:1022200012292B142C08013C031C3B294C3083162B
:10223000AC000A12831208230A1654308316AC002D
:102240000A12831208230A163D308316AC000A12C4
:10225000831208230A165C088316AA005730AB00C5
:102260000A12831264230A1620308316AC000A1265
:10227000831208230A16AF08031977290130E100F9
:102280000A122F270A1601308316A700D030A800A3
:102290000A1283120F230A168316A70183122F082E
:1022A0008316A8000A1283120F230A16AF01AB147B
:1022B0002C08033C031C5D292B142C08033C031C35
:1022C000762941308316AC000A12831208230A16BD
:1022D00053308316AC000A12831208230A162030EA
:1022E0008316AC000A12831208230A16BF2EB00808
:1022F0000319B42E2C08053C031C7F292B142C0831
:10230000053C031C982944308316AC000A12831242
:1023100008230A1652308316AC000A1283120823CF
:102320000A1620308316AC000A12831208230A16FC
:102330003008F700013077020319B3290230770221
:1023400003197D2A0330770203194C2B04307702DE
:1023500003191B2C053077020319EA2C063077028B
:102360000319B92D882E2C08053C031CB8292B1401
:102370002C08053C031CCD29E10161080A124A2101
:102380000A16E10AF7008316AC000A12831208232A
:102390000A1604306102031DBD292D082E02103CCF
:1023A0000318D4291030D6292D082E02E000AC08DD
:1023B000031DDB292B14AC08031DFF29E101610873
:1023C0000A1253210A16E10AF7008316AC000A121A
:1023D000831208230A1608306102031DDF296008F2
:1023E0008316AA005730AB000A12831264230A1620
:1023F00020308316AC000A12831208230A1601301B
:102400008316A700A8000A1283120F230A160130B0
:102410008316A700F030A8000A1283120F230A16B1
:102420008316A701A8010A1283120F230A16831626
:10243000A701831260088316A8000A1283120F23D3
:102440000A162D08E00760082D020318502A2C08F0
:10245000053C031C3F2A2D080A1233200A16E1000E
:102460008316AA005730AB000A12831264230A169F
:1024700020308316AC000A12831208230A162D0896
:102480000A1233200A16E1008316A701831261089D
:102490008316A8000A1283120F230A16AD0A232AF4
:1024A00001308316A700FA30A8000A1283120F2306
:1024B0000A162D08123C0319B001AB142C08023C7B
:1024C000031C632A2B142C08023C031C7C2A443076
:1024D0008316AC000A12831208230A16533083169F
:1024E000AC000A12831208230A1620308316AC00AF
:1024F0000A12831208230A16B32E2C08053C031C6B
:10250000822A2B142C08053C031C972AE101610840
:102510000A1263210A16E10AF7008316AC000A12B8
:10252000831208230A1604306102031D872A2D082E
:102530002E02103C03189E2A1030A02A2D082E02CD
:10254000E000AC08031DA52A2B14AC08031DC92A02
:10255000E10161080A1253210A16E10AF700831605
:10256000AC000A12831208230A1608306102031D08
:10257000A92A60088316AA005730AB000A128312FA
:1025800064230A1620308316AC000A128312082333
:102590000A1601308316A700A8000A1283120F231F
:1025A0000A1601308316A700F030A8000A12831221
:1025B0000F230A168316A701A8010A1283120F23FC
:1025C0000A168316A701831260088316A8000A1250
:1025D00083120F230A162D08E00760082D02031846
:1025E0001F2B2C08053C031CF62A2B142C08053C39
:1025F000031C0E2B2D080A1249200A16E10083162F
:10260000AA005730AB000A12831264230A16203046
:102610008316AC000A12831208230A162D080A1228
:1026200049200A16E1008316A70183126108831668
:10263000A8000A1283120F230A16AD0AED2A0130F0
:102640008316A700FA30A8000A1283120F230A1675
:102650002D08223C0319B001AB142C08023C031CCA
:10266000322B2B142C08023C031C4B2B44308316BA
:10267000AC000A12831208230A1653308316AC00EA
:102680000A12831208230A1620308316AC000A129D
:10269000831208230A16B32E2C08053C031C512B69
:1026A0002B142C08053C031C662BE10161080A125F
:1026B0006C210A16E10AF7008316AC000A12831295
:1026C00008230A1604306102031D562B2D082E0222
:1026D000103C03186D2B10306F2B2D082E02E000DC
:1026E000AC08031D742B2B14AC08031D982BE101BF
:1026F00061080A1253210A16E10AF7008316AC009A
:102700000A12831208230A1608306102031D782B6F
:1027100060088316AA005730AB000A1283126423A4
:102720000A1620308316AC000A12831208230A16F8
:1027300001308316A700A8000A1283120F230A167D
:1027400001308316A700F030A8000A1283120F236D
:102750000A168316A701A8010A1283120F230A166C
:102760008316A701831260088316A8000A12831239
:102770000F230A162D08E00760082D020318EE2B20
:102780002C08053C031CC52B2B142C08053C031CF2
:10279000DD2B2D080A126F200A16E1008316AA000D
:1027A0005730AB000A12831264230A1620308316B6
:1027B000AC000A12831208230A162D080A126F2091
:1027C0000A16E1008316A701831261088316A80088
:1027D0000A1283120F230A16AD0ABC2B013083168E
:1027E000A700FA30A8000A1283120F230A162D0838
:1027F000043C0319B001AB142C08023C031C012C4F
:102800002B142C08023C031C1A2C44308316AC00F9
:102810000A12831208230A1653308316AC000A12D8
:10282000831208230A1620308316AC000A12831282
:1028300008230A16B32E2C08053C031C202C2B144D
:102840002C08053C031C352CE10161080A126C219F
:102850000A16E10AF7008316AC000A128312082355
:102860000A1604306102031D252C2D082E02103C8F
:1028700003183C2C10303E2C2D082E02E000AC0832
:10288000031D432C2B14AC08031D672CE1016108C8
:102890000A1253210A16E10AF7008316AC000A1245
:1028A000831208230A1608306102031D472C6008B2
:1028B0008316AA005730AB000A12831264230A164B
:1028C00020308316AC000A12831208230A16013046
:1028D0008316A700A8000A1283120F230A160130DC
:1028E0008316A700F030A8000A1283120F230A16DD
:1028F0008316A701A8010A1283120F230A16831652
:10290000A701831260088316A8000A1283120F23FE
:102910000A162D08E00760082D020318BD2C2C08AC
:10292000053C031C942C2B142C08053C031CAC2CDC
:102930002D080A1277200A16E1008316AA005730E4
:10294000AB000A12831264230A1620308316AC00EF
:102950000A12831208230A162D080A1277200A1673
:10296000E1008316A701831261088316A8000A12EA
:1029700083120F230A16AD0A8B2C01308316A70091
:10298000FA30A8000A1283120F230A162D08763C8B
:102990000319B001AB142C08023C031CD02C2B14DF
:1029A0002C08023C031CE92C44308316AC000A12AC
:1029B000831208230A1653308316AC000A128312BE
:1029C00008230A1620308316AC000A12831208234B
:1029D0000A16B32E2C08053C031CEF2C2B142C08D4
:1029E000053C031C042DE10161080A126C210A1642
:1029F000E10AF7008316AC000A12831208230A16B4
:102A000004306102031DF42C2D082E02103C031823
:102A10000B2D10300D2D2D082E02E000AC08031DEB
:102A2000122D2B14AC08031D362DE10161080A128A
:102A300053210A16E10AF7008316AC000A1283122A
:102A400008230A1608306102031D162D600883163C
:102A5000AA005730AB000A12831264230A162030F2
:102A60008316AC000A12831208230A16013083165B
:102A7000A700A8000A1283120F230A16013083163A
:102A8000A700F030A8000A1283120F230A1683163B
:102A9000A701A8010A1283120F230A168316A701A1
:102AA000831260088316A8000A1283120F230A16E5
:102AB0002D08E00760082D0203188C2D2C08053C1A
:102AC000031C632D2B142C08053C031C7B2D2D08A7
:102AD0000A12F1200A16E1008316AA005730AB0053
:102AE0000A12831264230A1620308316AC000A12DD
:102AF000831208230A162D080A12F1200A16E10093
:102B00008316A701831261088316A8000A12831294
:102B10000F230A16AD0A5A2D01308316A700FA308A
:102B2000A8000A1283120F230A162D08463C031927
:102B3000B001AB142C08023C031C9F2D2B142C0855
:102B4000023C031CB82D44308316AC000A128312D9
:102B500008230A1653308316AC000A128312082386
:102B60000A1620308316AC000A12831208230A16B4
:102B7000B32E2C08053C031CBE2D2B142C08053C41
:102B8000031CD32DE10161080A126C210A16E10A27
:102B9000F7008316AC000A12831208230A160430C9
:102BA0006102031DC32D2D082E02103C0318DA2DDF
:102BB0001030DC2D2D082E02E000AC08031DE12DA5
:102BC0002B14AC08031D052EE10161080A125321E4
:102BD0000A16E10AF7008316AC000A1283120823D2
:102BE0000A1608306102031DE52D60088316AA004D
:102BF0005730AB000A12831264230A162030831662
:102C0000AC000A12831208230A1601308316A700AB
:102C1000A8000A1283120F230A1601308316A70098
:102C2000F030A8000A1283120F230A168316A70198
:102C3000A8010A1283120F230A168316A701831212
:102C400060088316A8000A1283120F230A162D08A3
:102C5000E00760082D0203185B2E2C08053C031CBE
:102C6000322E2B142C08053C031C4A2E2D080A1268
:102C70003E210A16E1008316AA005730AB000A1263
:102C8000831264230A1620308316AC000A128312C2
:102C900008230A162D080A123E210A16E10083169F
:102CA000A701831261088316A8000A1283120F235A
:102CB0000A16AD0A292E01308316A700FA30A800A3
:102CC0000A1283120F230A162D08083C0319B001BB
:102CD000AB142C08023C031C6E2E2B142C08023C57
:102CE000031C872E44308316AC000A12831208237B
:102CF0000A1653308316AC000A12831208230A16F0
:102D000020308316AC000A12831208230A16B32E51
:102D10002C08023C031C8D2E2B142C08023C031C97
:102D2000B22EE10161080A1275210A16E10AF700C4
:102D30008316AC000A12831208230A1604306102BB
:102D4000031D922E30088316AA005730AB000A12DA
:102D5000831264230A1629308316AC000A128312E8
:102D600008230A16B32EBF2EAB1CB82EAB10BF2EF5
:102D700001308316A5000A128312F6230A16202FAB
:102D8000DE1D202F2C08023C031CC72E2B142C0800
:102D9000023C031CE02E31308316AC000A12831271
:102DA00008230A1649308316AC000A12831208233E
:102DB0000A1620308316AC000A12831208230A1662
:102DC00001308316A7004330A8000A1283120F2394
:102DD0000A165C308316A0000130A1000A1283128B
:102DE00049230A162C08023C031CF72E2B142C082E
:102DF000023C031C202F4C308316AC000A128312B5
:102E000008230A1654308316AC000A1283120823D2
:102E10000A163D308316AC000A12831208230A16E4
:102E20005C088316AA005730AB000A128312642391
:102E30000A1620308316AC000A12831208230A16E1
:0A2E400000288B108A110A121D28C9
:02400E00F13F80
:00000001FF
